:100000000C94AC050C948C250C94B9250C94D40557
:100010000C94D4050C94D4050C94D4050C94D405FC
:100020000C94D4050C94D4050C94D4050C94D405EC
:100030000C94D4050C94D4050C94D4050C94D405DC
:100040000C94E6250C94D4050C94A9270C94FB275A
:100050000C94D4050C94D4050C94D4050C94D405BC
:100060000C94D4050C94D40500000000000000009E
:100070000000000000000000000000000000000080
:100080000000000000000000000000000000000070
:100090000000000000000000000000000000000060
:1000A0000000000000000000000000000000000050
:1000B0000000006070303070F0E0000000000000D0
:1000C000000000000080E0E0E0E0E0E0E0E0C0C030
:1000D000800000000000E0E0E08000000000000080
:1000E000000000C0E0E020000080C0C0E0E0E0E0F0
:1000F000E0E0C00000000080E0E0E0E0E0E0E0E000
:10010000C0C08000000080C0E0B89C868301000071
:100110000000000000000000F0FFFF1F00000000D2
:1001200001010307FFFFFC000000001FFFFFE000CC
:10013000000080E0F87E1F07030000001F7FFFF132
:10014000E1C08080000100000000F0FFFFBF808060
:100150008080C0C1E3FF7F3F000001010101010178
:100160000100000000000000000080FCFFFF87800D
:100170008080C0C0E0F0F87F3F0F03000000000067
:1001800007FFFFFCFC3F0F0301000000000080C0E0
:100190008080808081C3C7FFFF7C000080FCFFFF60
:1001A0000F0303030303030101000000000000002C
:1001B0000000000000000000000000000000030339
:1001C0000303030303030301010000000000000018
:1001D000000000000000030100000000000000001B
:1001E00000000103030303030303010100000000F7
:1001F00003030300000000000000000000000000F6
:1002000000000000000000000000000000000000EE
:1002100000000000000000000000000000000000DE
:1002200000000000000000000000000000000000CE
:1002300000000000000000000000000000000000BE
:1002400000000000000000000000000000000000AE
:10025000000000000000000000000000000000009E
:1002600000002110422063308440A550C660E77032
:10027000088129914AA16BB18CC1ADD1CEE1EFF1DA
:100280003112100273325222B5529442F772D66282
:10029000399318837BB35AA3BDD39CC3FFF3DEE32A
:1002A0006224433420040114E664C774A4448554D2
:1002B0006AA54BB528850995EEE5CFF5ACC58DD57A
:1002C0005336722611163006D776F6669556B44622
:1002D0005BB77AA719973887DFF7FEE79DD7BCC7CA
:1002E000C448E5588668A778400861180228233872
:1002F000CCC9EDD98EE9AFF9488969990AA92BB91A
:10030000F55AD44AB77A966A711A500A333A122AC1
:10031000FDDBDCCBBFFB9EEB799B588B3BBB1AAB69
:10032000A66C877CE44CC55C222C033C600C411C11
:10033000AEED8FFDECCDCDDD2AAD0BBD688D499DB9
:10034000977EB66ED55EF44E133E322E511E700E61
:100350009FFFBEEFDDDFFCCF1BBF3AAF599F788F09
:100360008891A981CAB1EBA10CD12DC14EF16FE1E9
:100370008010A100C230E320045025404670676021
:10038000B9839893FBA3DAB33DC31CD37FE35EF339
:10039000B1029012F322D232354214527762567271
:1003A000EAB5CBA5A89589856EF54FE52CD50DC589
:1003B000E234C324A01481046674476424540544C1
:1003C000DBA7FAB79987B8975FE77EF71DC73CD7D9
:1003D000D326F2369106B016576676761546345611
:1003E0004CD96DC90EF92FE9C899E9898AB9ABA929
:1003F0004458654806782768C018E1088238A32861
:100400007DCB5CDB3FEB1EFBF98BD89BBBAB9ABB78
:10041000754A545A376A167AF10AD01AB32A923AB0
:100420002EFD0FED6CDD4DCDAABD8BADE89DC98DC8
:10043000267C076C645C454CA23C832CE01CC10C00
:100440001FEF3EFF5DCF7CDF9BAFBABFD98FF89F18
:10045000176E367E554E745E932EB23ED10EF01E50
:100460000608205F0000000000000000002F0000D0
:1004700000000700070000147F147F1400242A7F67
:100480002A120023130864620036495522500000E6
:100490000503000000001C224100000041221C0056
:1004A0000014083E08140008083E0808000000A0D8
:1004B00060000008080808080000606000000020D4
:1004C00010080402003E5149453E0000427F4000B2
:1004D000004261514946002141454B310018141238
:1004E0007F10002745454539003C4A494930000105
:1004F0007109050300364949493600064949291E54
:1005000000003636000000005636000000081422B5
:1005100041000014141414140000412214080002B5
:100520000151090600324959513E007C1211127CDA
:10053000007F49494936003E41414122007F414107
:10054000221C007F49494941007F09090901003EF9
:100550004149497A007F0808087F0000417F410037
:10056000002040413F01007F08142241007F4040AD
:100570004040007F020C027F007F0408107F003E95
:100580004141413E007F09090906003E4151215E7B
:10059000007F091929460046494949310001017F78
:1005A0000101003F4040403F001F2040201F003F0E
:1005B0004038403F006314081463000708700807C0
:1005C00000615149454300007F414100AA55AA55A9
:1005D000AA55000041417F000004020102040040CE
:1005E000404040400000030500000020545454786F
:1005F000007F484444380038444444200038444490
:10060000487F00385454541800087E09010200182D
:10061000A4A4A47C007F080404780000447D40006A
:10062000004080847D00007F102844000000417F4E
:100630004000007C04180478007C0804047800382A
:100640004444443800FC242424180018242418FCB2
:10065000007C0804040800485454542000043F441B
:100660004020003C4040207C001C2040201C003CDE
:100670004030403C004428102844001CA0A0A07C2E
:10068000004464544C440000107C8200000000FFD1
:1006900000000000827C10000000060909060C1012
:1006A0002D0D000000808080808080000000000010
:1006B0000103030303030301000000000000000026
:1006C0000000000000000000000000C0C0000000AA
:1006D00000000000028686868686860200000000F2
:1006E00081C3C3C3C3C3C381000000FC7A060606EE
:1006F0000606067AFC00007EBCC0C0C0C0C0C0BCFC
:100700007E0000000000000000000078FC000000F7
:10071000000000000000003C7E000000028686868B
:100720008686867AFC00007EBDC3C3C3C3C3C38173
:1007300000000000028686868686867AFC0000001D
:1007400081C3C3C3C3C3C3BD7E0000FC7880808067
:1007500080808078FC000000010303030303033D55
:100760007E0000FC7A86868686868602000000006F
:1007700081C3C3C3C3C3C3BD7E0000FC7A86868623
:10078000868686020000007EBDC3C3C3C3C3C3BD4B
:100790007E000000020606060606067AFC0000003F
:1007A000000000000000003C7E0000FC7A86868687
:1007B0008686867AFC00007EBDC3C3C3C3C3C3BDA7
:1007C0007E0000FC7A8686868686867AFC0000009B
:1007D00081C3C3C3C3C3C3BD7E000E182D0D00006B
:1007E00000000000000000000000000000001038C1
:1007F0003838383838383810000000000000000061
:1008000000000000000000000000000000000000E8
:1008100000000000000000000000000000000000D8
:1008200000000000000000000040E0E04000000088
:100830000000000002060E0E0E0E0E0E0602000054
:1008400000001038383838383838381000000000C8
:1008500080C0E0E0E0E0E0E0C080000000FCFAF6EC
:100860000E0E0E0E0E0EF6FAFC0000EFC78300000F
:100870000000000083C7EF00007FBFDFE0E0E0E0A2
:10088000E0E0DFBF7F00000000000000000000008B
:10089000F0F8FC000000000000000000000083C72A
:1008A000EF00000000000000000000001F3F7F007C
:1008B000000002060E0E0E0E0E0EF6FAFC0000E010
:1008C000D0B83838383838383B170F00007FBFDFD2
:1008D000E0E0E0E0E0E0C0800000000002060E0E74
:1008E0000E0E0E0EF6FAFC000000103838383838BC
:1008F0003838BBD7EF00000080C0E0E0E0E0E0E087
:10090000DFBF7F0000FCF8F0000000000000F0F8FE
:10091000FC00000F173B383838383838BBD7EF00A9
:10092000000000000000000000001F3F7F0000FCEE
:10093000FAF60E0E0E0E0E0E06020000000F173B0A
:10094000383838383838B8D0E000000080C0E0E0EF
:10095000E0E0E0E0DFBF7F0000FCFAF60E0E0E0ED6
:100960000E0E0602000000EFD7BB38383838383892
:10097000B8D0E000007FBFDFE0E0E0E0E0E0DFBF14
:100980007F00000002060E0E0E0E0E0EF6FAFC00A0
:100990000000000000000000000083C7EF0000001E
:1009A00000000000000000001F3F7F0000FCFAF67E
:1009B0000E0E0E0E0E0EF6FAFC0000EFD7BB383806
:1009C00038383838BBD7EF00007FBFDFE0E0E0E029
:1009D000E0E0DFBF7F0000FCFAF60E0E0E0E0E0EFA
:1009E000F6FAFC00000F173B383838383838BBD7D8
:1009F000EF00000080C0E0E0E0E0E0E0DFBF7F006B
:100A000000000000240027002A000000000025004C
:100A100028002B0000000000230026002900040409
:100A20000404040404040202020202020303030396
:100A30000303010204081020408001020408102072
:100A4000010204081020000000070002010000035A
:100A50000406000000000000000000407A10F35A75
:100A600000A0724E18090010A5D4E80000E87648EE
:100A7000170000E40B54020000CA9A3B000000E19A
:100A8000F505000080969800000040420F0000002D
:100A9000A08601000000102700000000E80300000D
:100AA00000006400000000000A00000000000100D7
:100AB000000000002C76D888DC674F0823DFC1DFF8
:100AC000AE59E1B1B796E5E3E453C63AE6519976FB
:100AD00096E8E6C28426EB898C9B62ED407C6FFC35
:100AE000EFBC9C9F40F2BAA56FA5F490055A2AF777
:100AF0005C936B6CF9676DC11BFCE0E40D47FEF580
:100B000020E6B500D0ED902E0300943577050080E7
:100B1000841E080000204E0A000000C80C33333346
:100B2000330F986E12831141EF8D2114893BE655E6
:100B300016CFFEE6DB18D1844B381BF77C1D901DC9
:100B4000A4BBE424203284725E228100C9F124EC2B
:100B5000A1E53D27450E6A2911241FBECFEFD8E03D
:100B6000DEBFCDBF11E0A0E0B1E0ECE4F1E602C0F1
:100B700005900D92A432B107D9F717E0A4E2B1E0D5
:100B800001C01D92A232B107E1F71BE0C8E5DBE02E
:100B900004C02297FE010E946930C435D107C9F70D
:100BA0000E94C1290C94A4300C940000EF92FF9293
:100BB0000F931F93F22FF02E47FD02C0E4E001C017
:100BC000E4E1242F332727FD309537FF03C030950C
:100BD00021953F4F4F2D512F0F2FEE2E0E941606BD
:100BE0008F2D912F1F910F91FF90EF900895FB0192
:100BF000DC0102C001900D9241505040D8F7089599
:100C0000FB01DC0101900D920020E1F70895FB014A
:100C1000DC014150504048F001900D920020C9F78E
:100C200001C01D9241505040E0F70895A9E0B0E0A6
:100C3000ECE1F6E00C9471306A01122FA02EBE2C6C
:100C40002BE3201718F42CE3922E02C0902E9394DD
:100C5000AE014F5F5F4F27E0092D0E947807BC016E
:100C60008981E82EFF24C70189709070019711F4E3
:100C7000ADE209C0B1FE02C0ABE205C0B0FC02C0EB
:100C8000A0E001C0A0E2E3FE3BC0AA2311F423E0F0
:100C900001C024E0211710F020E002C0121B212F18
:100CA000EB2CB4FE02C0322F0AC0F601322F80E2D4
:100CB00002C0819331503323E1F7C20ED11CAA2325
:100CC00019F0F601A1936F01F6013196E2FE05C01D
:100CD0009EE4D6019C9381E404C09EE6D6019C93D9
:100CE00081E611968C9391833296DF01832F90E2F7
:100CF00002C09D9381508823E1F7E30FF11D40C0AE
:100D0000E2FE42C0AA2311F423E001C024E021172F
:100D100010F020E002C0121B212FEB2CB4FE02C009
:100D2000922F0AC0F601922F80E202C08193915067
:100D30009923E1F7C20ED11CAA2319F0F601A19361
:100D40006F01F6013196E2FE08C089E4D6018C936A
:100D50008EE411968C9386E407C089E6D6018C93C5
:100D60008EE611968C9386E681833296DF01892F79
:100D700020E202C02D9381508823E1F7E90FF11D95
:100D800010822EEF3FEFAFC0161617061CF041E0A1
:100D900050E003C0AB014F5F5F4FAA2019F480E021
:100DA00090E003C08A2D90E0019620E030E0AA2375
:100DB00011F021E030E0240F351F280F391F812F5B
:100DC00090E02817390714F020E002C0121B212FF1
:100DD0004B2D50E0CA0180719070B4FC0DC0B3FC83
:100DE0000BC0F601322F40E202C041933150332351
:100DF000E1F7C20ED11C01C0322FAA2319F0F6016F
:100E0000A1936F01892B11F0132F0AC0F601132F44
:100E100080E302C0819311501123E1F7C30ED11C6E
:100E2000092D060FBA8090E1892E912C8E209F20EB
:100E3000E4FE04C0F1E3BF1609F40150101614F0EB
:100E400001E003C0093008F008E09B0177FF02C011
:100E500020E030E0CB010196821B930BFE0131961E
:100E6000E80FF91F8EE2F82E3B01601A71088A2DF7
:100E700090E044275527481B590B8FEF2F3F380729
:100E800019F4D601FD926D01621773072CF06216FA
:100E9000730614F4808101C080E321503040319604
:100EA0002417350724F0D6018D936D01E6CF261760
:100EB000370749F4B5E3BB1528F0BB1621F48114BC
:100EC000910409F481E3F6018193D601812F90E228
:100ED00002C09C93815011968823D9F7E10FF11D30
:100EE000108220E030E0C9012996EEE00C948D30AC
:100EF000283008F027E03327DA01990F311D87FDEC
:100F0000916000966105710539F432602E5F3D9362
:100F100030E32A95E1F708959F3F30F0803871055E
:100F2000610509F03C5F3C5F3D93913008F08068BB
:100F3000911DDF93CF931F930F93FF92EF92192F81
:100F4000987F9695E92F96959695E90FFF27EC5493
:100F5000F54F99273327EE24FF24A701E7010590D9
:100F60000894079428F4360FE71EF81E491F511DF8
:100F7000660F771F881F991F0694A1F705900794A5
:100F800028F4E70EF81E491F561FC11D770F881F52
:100F9000991F661F0694A1F70590079428F4F80E90
:100FA000491F561FC71FD11D880F991F661F771F26
:100FB0000694A1F70590079420F4490F561FC71F08
:100FC000D81F990F661F771F881F0694A9F7849171
:100FD0001095177041F0D695C79557954795F7949A
:100FE000E7941A95C1F7EAE5FAE06894159015912F
:100FF00035916591959105907FE27395E118F10A1D
:10100000430B560BC90BD009C0F7E10CF11E431F6F
:10101000561FC91FD01D7EF4703311F48A95E6CF98
:10102000E894015030F0080F0AF40027021708F482
:10103000202F2395022F7A3328F079E37D932A9588
:10104000E9F710C07D932A9589F6069497956795E0
:10105000379517951794E118F10A430B560BC90BF6
:10106000D00998F023957E9173957A3308F070E358
:101070007C932013B8F77E9170617D9330F0839557
:1010800071E37D9370E32A95E1F71124EF90FF90CF
:101090000F911F91CF91DF91992787FD909508952A
:1010A00061E070E040E050E016C0342F2227FB01E1
:1010B000E75AFA4F8081E82FF0E0852F9927E8273B
:1010C000F927EE0FFF1FE05AFD4F4591549142273B
:1010D00053276F5F7F4F80919105909192058617FE
:1010E00097071CF74093A9055093AA05E091910535
:1010F000F0919205E55AFA4F4083E0919105F09105
:101100009205E65AFA4F508380919105909192058D
:10111000029690939205809391050895AF92BF92A5
:10112000CF92DF92EF92FF920F931F93CF93DF93B3
:101130001092EE041092ED048FEF8093F104109260
:10114000F0041092EF048AEE8093270186EA8093E0
:1011500028011092290184E090E090937E0480930E
:101160007D0483E090E09093800480937F0440E0CE
:1011700050E0C1E0D0E031E0E32EF12C012D112D43
:101180001092F0041092EF04BE01042E02C0660F0C
:10119000771F0A94E2F766C08091EF049091F00403
:1011A000FC01EE0FFF1FE80FF91FE756FB4F808190
:1011B00090E086239723892BB9F0E0917F04F0918A
:1011C0008004EA5DFE4F208180917D0490917E0431
:1011D0005701680104C0AA0CBB1CCC1CDD1C8A95FD
:1011E000D2F72A29208319C0E0917F04F09180046E
:1011F000EA5DFE4F208180917D0490917E0457012D
:10120000680104C0AA0CBB1CCC1CDD1C8A95D2F75B
:10121000D601C50180958223808380917D049091C1
:101220007E04019690937E0480937D0480917D04DA
:1012300090917E0408976CF010927E0410927D04C9
:1012400080917F0490918004019690938004809314
:101250007F048091EF049091F00401969093F00444
:101260008093EF048091EF049091F0044C970CF47C
:1012700093CF4F5F5F4F4830510509F081CF40E079
:1012800050E0C1E0D0E0B1E0EB2EF12C012D112DAA
:101290001092F0041092EF04BE01042E02C0660FFB
:1012A000771F0A94E2F766C08091EF049091F004F2
:1012B000FC01EE0FFF1FE80FF91FE756FB4F81817E
:1012C00090E086239723892BB9F0E0917F04F09179
:1012D0008004EA5DFE4F208180917D0490917E0420
:1012E0005701680104C0AA0CBB1CCC1CDD1C8A95EC
:1012F000D2F72A29208319C0E0917F04F09180045D
:10130000EA5DFE4F208180917D0490917E0457011B
:10131000680104C0AA0CBB1CCC1CDD1C8A95D2F74A
:10132000D601C50180958223808380917D049091B0
:101330007E04019690937E0480937D0480917D04C9
:1013400090917E0408976CF010927E0410927D04B8
:1013500080917F0490918004019690938004809303
:101360007F048091EF049091F00401969093F00433
:101370008093EF048091EF049091F0044C970CF46B
:1013800093CF4F5F5F4F4430510509F081CF44E068
:1013900050E0C1E0D0E031E0E32EF12C012D112D21
:1013A0001092F0041092EF04BE01042E02C0660FEA
:1013B000771F0A94E2F766C08091EF049091F004E1
:1013C000FC01EE0FFF1FE80FF91FE756FB4F81816D
:1013D00090E086239723892BB9F0E0917F04F09168
:1013E0008004EA5DFE4F208180917D0490917E040F
:1013F0005701680104C0AA0CBB1CCC1CDD1C8A95DB
:10140000D2F72A29208319C0E0917F04F09180044B
:10141000EA5DFE4F208180917D0490917E0457010A
:10142000680104C0AA0CBB1CCC1CDD1C8A95D2F739
:10143000D601C50180958223808380917D0490919F
:101440007E04019690937E0480937D0480917D04B8
:1014500090917E0408976CF010927E0410927D04A7
:1014600080917F04909180040196909380048093F2
:101470007F048091EF049091F00401969093F00422
:101480008093EF048091EF049091F0044B970CF45B
:1014900093CF4F5F5F4F4830510509F081CF40E057
:1014A00050E0C1E0D0E0B1E0EB2EF12C012D112D88
:1014B0001092F0041092EF04BE01042E02C0660FD9
:1014C000771F0A94E2F766C08091EF049091F004D0
:1014D000FC01EE0FFF1FE80FF91FE756FB4F82815B
:1014E00090E086239723892BB9F0E0917F04F09157
:1014F0008004EA5DFE4F208180917D0490917E04FE
:101500005701680104C0AA0CBB1CCC1CDD1C8A95C9
:10151000D2F72A29208319C0E0917F04F09180043A
:10152000EA5DFE4F208180917D0490917E045701F9
:10153000680104C0AA0CBB1CCC1CDD1C8A95D2F728
:10154000D601C50180958223808380917D0490918E
:101550007E04019690937E0480937D0480917D04A7
:1015600090917E0408976CF010927E0410927D0496
:1015700080917F04909180040196909380048093E1
:101580007F048091EF049091F00401969093F00411
:101590008093EF048091EF049091F0044B970CF44A
:1015A00093CF4F5F5F4F4830510509F081CF84E002
:1015B00090E090937E0480937D0483E090E090938C
:1015C000800480937F0481E090E09093F004809306
:1015D000EF0441E0E42EF12C012D112D8EC08091FD
:1015E000F104880F8093F1048091F1042091F104BB
:1015F00090E034E0959587953A95E1F78170907089
:10160000221F2227221F30E08217930721F08091AA
:10161000F104816003C08091F1048E7F8093F10416
:101620002091F104E0917F04F0918004EA5DFE4F87
:10163000808140917D0450917E0490E002C0959598
:1016400087954A95E2F730E08227932780FF17C0FD
:10165000E0917F04F0918004EA5DFE4F208180914B
:101660007D0490917E04B801A70104C0440F551F6A
:10167000661F771F8A95D2F7242B208319C0E0912B
:101680007F04F0918004EA5DFE4F208180917D040B
:1016900090917E045701680104C0AA0CBB1CCC1CAD
:1016A000DD1C8A95D2F7D601C501809582238083FF
:1016B00080917D0490917E04019690937E048093A6
:1016C0007D0480917D0490917E0408976CF01092C7
:1016D0007E0410927D0480917F0490918004019695
:1016E0009093800480937F048091EF049091F004A4
:1016F00001969093F0048093EF048091EF04909111
:10170000F004855992400CF46ACFDF91CF911F917C
:101710000F91FF90EF90DF90CF90BF90AF90089522
:101720004091F1042091F1048091F10430E035956D
:10173000279550E0422753274170507090E09595CF
:10174000879595958795817090704817590709F18D
:101750008091EE042091ED0490E0FC01EE0FFF1F5C
:10176000E80FF91FE20FF11DE756FB4F4081209172
:10177000EF043091F00481E090E0A0E0B0E004C01C
:10178000880F991FAA1FBB1F2A95D2F7482B4083A9
:1017900021C08091EE042091ED0490E0FC01EE0F59
:1017A000FF1FE80FF91FE20FF11DE756FB4F4081C5
:1017B0002091EF043091F00481E090E0A0E0B0E0EF
:1017C00004C0880F991FAA1FBB1F2A95D2F78095C6
:1017D000842380838091EF049091F004019690938C
:1017E000F0048093EF042091F1048091F10490E0E3
:1017F000959587959595879530E08227932780FF6B
:1018000021C08091EE042091ED0490E0FC01EE0FE8
:10181000FF1FE80FF91FE20FF11DE756FB4F408154
:101820002091EF043091F00481E090E0A0E0B0E07E
:1018300004C0880F991FAA1FBB1F2A95D2F7482BF7
:10184000408321C08091EE042091ED0490E0FC01E2
:10185000EE0FFF1FE80FF91FE20FF11DE756FB4FD8
:1018600040812091EF043091F00481E090E0A0E00D
:10187000B0E004C0880F991FAA1FBB1F2A95D2F79A
:101880008095842380838091EF049091F0040196E9
:101890009093F0048093EF040895CF93DF93109218
:1018A000EE041092ED041092F1041092F0041092E4
:1018B000EF0481E090E045C0C0E0D0E08091F10409
:1018C000880F8093F104E0911D05F0911E05EE5004
:1018D000FB4F808190E00C2E02C0959587950A946D
:1018E000E2F780FF04C08091F104816003C0809121
:1018F000F1048E7F8093F1040E94900B8091EF049D
:101900009091F0040897A4F01092F0041092EF0464
:101910008091ED048F5F8093ED048091ED0483301E
:1019200038F01092ED048091EE048F5F8093EE0406
:101930002196C830D10511F680911D0590911E05A4
:10194000019690931E0580931D0580911D05909131
:101950001E058A970CF4B0CF8091F104880F809314
:10196000F1048091F1048E7F8093F1040E94900B2A
:101970008091F104880F8093F1048091F1048E7FAF
:101980008093F1040E94900BDF91CF910895809194
:10199000F10483FFC6C08091F10486FFC2C004C079
:1019A0008091F10486FDC1C08091F104880F80937D
:1019B000F1048091F1048E7F8093F10480918B0477
:1019C00080FFBCC08091F10480FFB8C004C080914A
:1019D000F10480FDB7C08091EE042091ED0490E009
:1019E000FC01EE0FFF1FE80FF91FE20FF11DE75694
:1019F000FB4F40812091EF043091F00481E090E0B2
:101A0000A0E0B0E004C0880F991FAA1FBB1F2A9551
:101A1000D2F78095842380838091EE048F5F80933A
:101A2000EE048091ED04882301F58091EE048C3161
:101A3000E0F01092EE048091EF049091F004019791
:101A40009093F0048093EF048091EF049091F00460
:101A500097FF0BC087E090E09093F0048093EF0431
:101A60008091ED048F5F8093ED048091ED048130CF
:101A700079F48091EE048C3158F01092EE0480914C
:101A8000EF049091F00401979093F0048093EF0499
:101A90008091ED048130A9F48091EE048B3189F4BA
:101AA0008091EF049091F00404975CF41092EE049E
:101AB0008091EF049091F00401979093F00480934B
:101AC000EF048091EF049091F00497FF0BC087E042
:101AD00090E09093F0048093EF048091ED048F5F89
:101AE0008093ED048091ED04823009F04CC0809128
:101AF000EE048B3108F447C01092EE048091EF049D
:101B00009091F00401979093F0048093EF048091FA
:101B1000EF049091F00497FF36C083E08093960520
:101B200008958091F10483FF3BCF8091F104880FE9
:101B30008093F1048091F10481603ECF80918B0409
:101B400080FF45CF8091EE042091ED0490E0FC01F0
:101B5000EE0FFF1FE80FF91FE20FF11DE756FB4FD5
:101B600040812091EF043091F00481E090E0A0E00A
:101B7000B0E004C0880F991FAA1FBB1F2A95D2F797
:101B8000482B408349CF08958091F10487FF19C005
:101B90008091F10482FF15C004C08091F10482FDA0
:101BA00014C08091F1048E7F8093F10480911C0514
:101BB00090E09595879580931C0580911C058F7703
:101BC00013C08091F10487FFE8CF8091F104816018
:101BD0008093F10480911C0590E095958795809302
:101BE0001C0580911C05806880931C058091F10480
:101BF000880F8093F1040895809198048F5F8093FB
:101C0000980480919804883000F110929804E09133
:101C10000701F0910801EA5DFE4F80818093810405
:101C2000809107019091080101979093080180939A
:101C300007018091070190910801892B31F48CE212
:101C400091E09093080180930701E6E1F0E0DF0165
:101C5000AF57BB4F8C9190E0959587958C939F01E2
:101C600021503040F901EF57FB4F808180FF03C0C6
:101C70008C91806802C08C918F778C938FEF2F3F6F
:101C8000380711F0F901E3CF0895EF92FF920F9317
:101C90001F938CEC95E06EE070E04FE050E020E1A7
:101CA00030E002E110E0E1E1EE2EF12C0E941D2473
:101CB0001F910F91FF90EF9008952F923F924F92B6
:101CC0005F926F927F928F929F92AF92BF92CF92CC
:101CD000DF92EF92FF920F931F93DF93CF93CDB7D5
:101CE000DEB7CE54D0400FB6F894DEBF0FBECDBFE6
:101CF00020E030E095E2E92EF12CEC0EFD1EBE0155
:101D0000625D7F4F87E3482E512C4C0E5D1E00E430
:101D1000202E312C2C0E3D1EF901EA50FB4F808104
:101D2000F701E20FF31F8083F901E250FB4F80813E
:101D3000FB01E20FF31F8083F901EA5FFA4F808114
:101D4000F201E20FF31F8083F901E25FFA4F808115
:101D5000F101E20FF31F80832F5F3F4F28303105E1
:101D6000D9F68FE2FE01E85BFF4F80838091160574
:101D7000FE01E75BFF4F808380911705FE01E65B64
:101D8000FF4F808380911805FE01E55BFF4F808344
:101D900080911905FE01E45BFF4F80831DA61EAAFA
:101DA0001FAEFE01E35BFF4F10823E010894611CF1
:101DB000711CC3010E94F12A17E0812E912C8C0E18
:101DC0009D1EC401B30140E050E028E030E00E94D5
:101DD000232BBDE0AB2EB12CAC0EBD1EC501B40152
:101DE0000E948B2BC50160E071E00E949E2A8C014D
:101DF000A3E1CA2ED12CCC0EDD1EC601B7010E9474
:101E0000F12AF9E1EF2EF12CEC0EFD1EC701B6010F
:101E100047E050E028E030E00E94232BC801B701E2
:101E20000E94BA2ABC018E01015E1F4FC8010E94A8
:101E3000812B8CEC95E0B80140E050E028E130E0E7
:101E40000E945523C8010E94952BC7010E94952B23
:101E5000C6010E94952BC5010E949B2BC4010E94C4
:101E6000952BC3010E94952B8CEC95E0B20140E0CC
:101E700050E020E230E00E94D9228CEC95E0B101E4
:101E800040E050E028E230E00E94D922C25BDF4F00
:101E90000FB6F894DEBF0FBECDBFCF91DF911F917B
:101EA0000F91FF90EF90DF90CF90BF90AF909F90F9
:101EB0008F907F906F905F904F903F902F900895FC
:101EC0002F923F924F925F926F927F928F929F924A
:101ED000AF92BF92CF92DF92EF92FF920F931F9338
:101EE000DF93CF93CDB7DEB7CE54D0400FB6F89482
:101EF000DEBF0FBECDBF20E030E0A5E2EA2EF12C20
:101F0000EC0EFD1EBE01625D7F4FF7E34F2E512C9C
:101F10004C0E5D1EE0E42E2E312C2C0E3D1EF901E0
:101F2000EB50FB4F8081F701E20FF31F8083F90133
:101F3000E350FB4F8081FB01E20FF31F8083F90127
:101F4000EB5FFA4F8081F201E20FF31F8083F9010A
:101F5000E35FFA4F8081F101E20FF31F80832F5F6F
:101F60003F4F28303105D9F68FE2FE01E85BFF4F85
:101F7000808380911505FE01E75BFF4F8083809190
:101F80001605FE01E65BFF4F808380911705FE0179
:101F9000E55BFF4F808380911805FE01E45BFF4FF6
:101FA00080831DA61EAA1FAEFE01E35BFF4F1082B9
:101FB0003E010894611C711CC3010E94F12A57E084
:101FC000852E912C8C0E9D1EC401B30140E050E083
:101FD00028E030E00E94232B4DE0A42EB12CAC0E63
:101FE000BD1EC501B4010E948B2BC50160E071E0EC
:101FF0000E949E2A8C0133E1C32ED12CCC0EDD1E13
:10200000C601B7010E94F12A29E1E22EF12CEC0E63
:10201000FD1EC701B60147E050E028E030E00E9415
:10202000232BC801B7010E94BA2ABC018E01015EB0
:102030001F4FC8010E94812B8CEC95E0B80140E055
:1020400050E028E130E00E945523C8010E94952B02
:10205000C7010E94952BC6010E94952BC5010E94C5
:102060009B2BC4010E94952BC3010E94952B8CECE5
:1020700095E0B20140E050E020E230E00E94D92239
:102080008CEC95E0B10140E050E028E230E00E94A5
:10209000D922C25BDF4F0FB6F894DEBF0FBECDBFB3
:1020A000CF91DF911F910F91FF90EF90DF90CF9034
:1020B000BF90AF909F908F907F906F905F904F9068
:1020C0003F902F90089580910A0190910B010E94FA
:1020D0005527019749F480910C0190910D010E94C0
:1020E0005527892B49F415C080910C0190910D0161
:1020F0000E945527892B69F48091B3059091B4050E
:10210000A091B505B091B6058C529F4CAF4FBF4F13
:102110000CC08091B3059091B405A091B505B09124
:10212000B605845D9043A040B0408093B305909382
:10213000B405A093B505B093B60508958091AB059D
:102140009091AC0501969093AC058093AB0585E02A
:102150000E945527892B21F080912401806803C0BB
:10216000809124018F7780932401809125018F5FD6
:102170008093250180912501883009F5E0910501C2
:10218000F091060180912401EA5DFE4F80838091E9
:102190000501909106010197909306018093050136
:1021A0008091050190910601892B31F48CE291E038
:1021B00090930601809305011092250107C080913C
:1021C000240190E0959587958093240181E0809388
:1021D00098050895EF92FF920F931F936091B305B6
:1021E0007091B4058091B5059091B60564527C4B11
:1021F000814090400E94B62E28EA3DEF40EE5AE41E
:102200000E94202E6093B7057093B8058093B9059E
:102210009093BA056091B7057091B8058091B905A2
:102220009091BA050E94F12E0E94882E6093BB0502
:10223000E090B705F090B8050091B9051091BA0586
:102240006091BB0570E0882777FD8095982F0E94EC
:10225000B62E9B01AC01C801B7010E94B72D20E04A
:1022600030E040E057E40E94BB2F6093B7057093C5
:10227000B8058093B9059093BA056091B705709140
:10228000B8058091B9059091BA0520E030E040E0B2
:102290005FE30E94B82D0E94F12E0E94882E709359
:1022A000BD056093BC0583E090E0A0E0B0E08093C2
:1022B000BE059093BF05A093C005B093C105809162
:1022C000BE059091BF05A091C005B091C105BA2F80
:1022D000A92F982F88278093BE059093BF05A093C0
:1022E000C005B093C1052091BE053091BF05409156
:1022F000C0055091C1058091BB0590E0A0E0B0E021
:10230000822B932BA42BB52B8093BE059093BF05F6
:10231000A093C005B093C1058091BE059091BF0503
:10232000A091C005B091C1054FE0880F991FAA1F69
:10233000BB1F4A95D1F78093BE059093BF05A0932C
:10234000C005B093C1052091BE053091BF054091F5
:10235000C0055091C1058091BC059091BD05A0E0DC
:10236000B0E0822B932BA42BB52B8093BE059093CA
:10237000BF05A093C005B093C1058091BE059091A3
:10238000BF05A091C005B091C10534E0880F991F29
:10239000AA1FBB1F3A95D1F78093BE059093BF0546
:1023A000A093C005B093C1056091B3057091B405C9
:1023B0008091B5059091B605645875438040904072
:1023C0000E94B62E28EA3DEF40EE5AE40E94202EED
:1023D0006093B7057093B8058093B9059093BA05DB
:1023E0006091B7057091B8058091B9059091BA05D3
:1023F0000E94F12E0E94882E6093BB05E090B705E5
:10240000F090B8050091B9051091BA056091BB052F
:1024100070E0882777FD8095982F0E94B62E9B014B
:10242000AC01C801B7010E94B72D20E030E040E0C8
:1024300057E40E94BB2F6093B7057093B805809353
:10244000B9059093BA056091B7057091B805809170
:10245000B9059091BA0520E030E040E05FE30E94CA
:10246000B82D0E94F12E0E94882E7093BD056093B6
:10247000BC0582E090E0A0E0B0E08093C2059093BC
:10248000C305A093C405B093C5058091C205909182
:10249000C305A091C405B091C505BA2FA92F982FE7
:1024A00088278093C2059093C305A093C405B09379
:1024B000C5052091C2053091C3054091C4055091D6
:1024C000C5058091BB0590E0A0E0B0E0822B932B86
:1024D000A42BB52B8093C2059093C305A093C4058C
:1024E000B093C5058091C2059091C305A091C40524
:1024F000B091C5050FE0880F991FAA1FBB1F0A9551
:10250000D1F78093C2059093C305A093C405B093FF
:10251000C5052091C2053091C3054091C405509175
:10252000C5058091BC059091BD05A0E0B0E0822B6F
:10253000932BA42BB52B8093C2059093C305A09336
:10254000C405B093C5058091C2059091C305A091C3
:10255000C405B091C50514E0880F991FAA1FBB1FC1
:102560001A95D1F78093C2059093C305A093C40533
:10257000B093C5051F910F91FF90EF900895EF92D2
:10258000FF920F931F938091260590E09093C705CB
:102590008093C6058091C6059091C705A0E0B0E084
:1025A0008093B3059093B405A093B505B093B60599
:1025B0008091270590E09093C7058093C6052091F0
:1025C000B3053091B4054091B5055091B6058091A1
:1025D000C6059091C705982F8827A0E0B0E0820F2C
:1025E000931FA41FB51F8093B3059093B405A093C8
:1025F000B505B093B6058091280590E09093C70586
:102600008093C6052091B3053091B4054091B5057E
:102610005091B6058091C6059091C705A0E0B0E045
:10262000DC0199278827820F931FA41FB51F809371
:10263000B3059093B405A093B505B093B60580910A
:10264000290590E09093C7058093C6052091B305B6
:102650003091B4054091B5055091B6058091C605FD
:102660009091C705A0E0B0E0B82FAA279927882746
:10267000820F931FA41FB51F8093B3059093B405D9
:10268000A093B505B093B6056091B3057091B405FC
:102690008091B5059091B60564527C4B8140904085
:1026A0000E94B62E28EA3DEF40EE5AE40E94202E0A
:1026B0006093B7057093B8058093B9059093BA05F8
:1026C0006091B7057091B8058091B9059091BA05F0
:1026D0000E94F12E0E94882E6093BB05E090B70502
:1026E000F090B8050091B9051091BA056091BB054D
:1026F00070E0882777FD8095982F0E94B62E9B0169
:10270000AC01C801B7010E94B72D20E030E040E0E5
:1027100057E40E94BB2F6093B7057093B805809370
:10272000B9059093BA056091B7057091B80580918D
:10273000B9059091BA0520E030E040E05FE30E94E7
:10274000B82D0E94F12E0E94882E7093BD056093D3
:10275000BC0583E090E0A0E0B0E08093BE059093DC
:10276000BF05A093C005B093C1058091BE059091AF
:10277000BF05A091C005B091C105BA2FA92F982F10
:1027800088278093BE059093BF05A093C005B093A2
:10279000C1052091BE053091BF054091C005509103
:1027A000C1058091BB0590E0A0E0B0E0822B932BA7
:1027B000A42BB52B8093BE059093BF05A093C005B5
:1027C000B093C1058091BE059091BF05A091C00551
:1027D000B091C1051FE0880F991FAA1FBB1F1A9552
:1027E000D1F78093BE059093BF05A093C005B09329
:1027F000C1052091BE053091BF054091C0055091A3
:10280000C1058091BC059091BD05A0E0B0E0822B90
:10281000932BA42BB52B8093BE059093BF05A0935B
:10282000C005B093C1058091BE059091BF05A091F0
:10283000C005B091C105F4E0880F991FAA1FBB1F06
:10284000FA95D1F78093BE059093BF05A093C0057C
:10285000B093C1056091B3057091B4058091B50541
:102860009091B60564587543804090400E94B62E02
:1028700028EA3DEF40EE5AE40E94202E6093B7050F
:102880007093B8058093B9059093BA056091B70528
:102890007091B8058091B9059091BA050E94F12E0A
:1028A0000E94882E6093BB05E090B705F090B805B4
:1028B0000091B9051091BA056091BB0570E08827B9
:1028C00077FD8095982F0E94B62E9B01AC01C80120
:1028D000B7010E94B72D20E030E040E057E40E94AD
:1028E000BB2F6093B7057093B8058093B90590939B
:1028F000BA056091B7057091B8058091B9059091BE
:10290000BA0520E030E040E05FE30E94B82D0E946D
:10291000F12E0E94882E7093BD056093BC0582E065
:1029200090E0A0E0B0E08093C2059093C305A0932F
:10293000C405B093C5058091C2059091C305A091CF
:10294000C405B091C505BA2FA92F982F8827809369
:10295000C2059093C305A093C405B093C50520910B
:10296000C2053091C3054091C4055091C5058091C1
:10297000BB0590E0A0E0B0E0822B932BA42BB52BFD
:102980008093C2059093C305A093C405B093C50579
:102990008091C2059091C305A091C405B091C50571
:1029A0007FE0880F991FAA1FBB1F7A95D1F78093EC
:1029B000C2059093C305A093C405B093C5052091AB
:1029C000C2053091C3054091C4055091C505809161
:1029D000BC059091BD05A0E0B0E0822B932BA42B09
:1029E000B52B8093C2059093C305A093C405B09303
:1029F000C5058091C2059091C305A091C405B09111
:102A0000C50564E0880F991FAA1FBB1F6A95D1F7FF
:102A10008093C2059093C305A093C405B093C505E8
:102A20001F910F91FF90EF9008958091AB059091C9
:102A3000AC0501969093AC058093AB058091A00501
:102A40009091A10501979093A1058093A005809195
:102A50009905843021F080919905853009F510920F
:102A6000A7051092A6058091A80581508093A8051E
:102A700086E00E945527019719F486E060E002C0C5
:102A800086E061E00E94012780919905853041F43C
:102A900086E00E945527019719F486E080939905F6
:102AA00080919905873029F080919905883009F047
:102AB00070C08091A6059091A70501969093A705F7
:102AC0008093A6058091A6059091A7058036910573
:102AD0005CF01092A7051092A6058091A5058F5F66
:102AE0008093A5058091A505E0917B04F0917C047D
:102AF000EA5DFE4F808120917D0430917E0490E05C
:102B000002C0959587952A95E2F780FF03C086E07D
:102B100061E002C086E060E00E94012780917D04B0
:102B200090917E04019690937E0480937D04809121
:102B30007D0490917E040897D1F410927E04109247
:102B40007D0480917B0490917C04019690937C0499
:102B500080937B0480917B0490917C048355934007
:102B600034F081E090E090937C0480937B0480912A
:102B70009905883071F42091790430917A0480911C
:102B80007B0490917C042817390719F489E080931D
:102B9000990581E080939B0583E160E00E94012715
:102BA00008958FE190E029C08091AD059091AE0528
:102BB000A091AF05B091B0052091B1053091B2055B
:102BC00004C0B595A795979587952A95D2F780FF6C
:102BD00003C08AE061E002C08AE060E00E94012751
:102BE00087E061E00E94012787E060E00E94012702
:102BF0008091B1059091B20501979093B2058093B1
:102C0000B1058091B1059091B20597FFCDCF8CE0D1
:102C100061E00E9401278CE060E00E9401278AE0C9
:102C200060E00E940127089585EF94E2A0E0B0E003
:102C30008093AD059093AE05A093AF05B093B0051A
:102C40000E94D11582E990EDA5E6B1E08093AD0533
:102C50009093AE05A093AF05B093B0050E94D11537
:102C600083E990ECACE4BAE28093AD059093AE05B5
:102C7000A093AF05B093B0050E94D11584E194EC08
:102C8000A5E4B0E48093AD059093AE05A093AF05A5
:102C9000B093B0050E94D1158091BE059091BF05FB
:102CA000A091C005B091C1058093AD059093AE058C
:102CB000A093AF05B093B0050E94D115089582E9A5
:102CC00090EDA5E7B0E08093AD059093AE05A0939D
:102CD000AF05B093B0050E94D1158091C2059091C7
:102CE000C305A091C405B091C5058093AD0590932F
:102CF000AE05A093AF05B093B0050E94D11508951D
:102D000081E190E5A7E5B0E08093AD059093AE0535
:102D1000A093AF05B093B0050E94D11583E990EC64
:102D2000ACE4BAE28093AD059093AE05A093AF05F5
:102D3000B093B0050E94D1158091BE059091BF055A
:102D4000A091C005B091C1058093AD059093AE05EB
:102D5000A093AF05B093B0050E94D11585EF94E222
:102D6000A0E0B0E08093AD059093AE05A093AF05D1
:102D7000B093B0050E94D11584E194ECA5E4B0E4D1
:102D80008093AD059093AE05A093AF05B093B005C9
:102D90000E94D11582E990EDA5E6B1E08093AD05E2
:102DA0009093AE05A093AF05B093B0050E94D115E6
:102DB0008FE090E0AEE0B0E08093AD059093AE057B
:102DC000A093AF05B093B0050E94D11586E09EE0B8
:102DD000A7E0B5E08093AD059093AE05A093AF0555
:102DE000B093B0050E94D11589EE91E3A2E0B0E066
:102DF0008093AD059093AE05A093AF05B093B00559
:102E00000E94D1158AE397E4A6E9B2E38093AD0569
:102E10009093AE05A093AF05B093B0050E94D11575
:102E20008BE390E0A0E0B0E08093AD059093AE0519
:102E3000A093AF05B093B0050E94D1158CE091E04E
:102E4000A0E0B0E08093AD059093AE05A093AF05F0
:102E5000B093B0050E94D1158DE090E0A0E0B0E005
:102E60008093AD059093AE05A093AF05B093B005E8
:102E70000E94D115089580E48093260588E7809309
:102E8000270587EE8093280589E1809329050E9414
:102E9000BF120E94801680E00E94792580E06EE9D2
:102EA00070E143E050E00E945625089580E00E94C2
:102EB000792580E06EE970E143E050E00E945625FC
:102EC00081E00E94792581E063E670E143E050E013
:102ED0000E9456258091A3058E7F8093A305809143
:102EE000A3058D7F8093A30588E060E00E94012701
:102EF0008DE060E00E9401270E9414168CE291E0B0
:102F00009093060180930501109298041092960503
:102F100010929305109294051092A5051092A405A5
:102F200081E08093990510929A0580939705089502
:102F3000CF93DF9380ED80935A050E945008C1E043
:102F4000D0E009C0FE01E75AFA4F60818CEF96E0AD
:102F50000E942A29219680919105909192058C17C3
:102F60009D0784F7DF91CF910895FF920F931F93F0
:102F700080918F048A3A09F050C080918E048A3A79
:102F800009F04BC080918D048E3609F046C08091C7
:102F90008C048A3009F041C082E08093960510923B
:102FA000ED041092EE0487E090E09093F00480939B
:102FB000EF048FEF8093F104109295058091090141
:102FC0008F5F80930901F3E0FF2EF0925B05109272
:102FD0005C0585E180935D0510925E0510925F05AA
:102FE00006E010E010939205009391050E94981757
:102FF000F0925B0510925C0586E180935D058091FF
:10300000090180935E058091950580935F0510937B
:103010009205009391050E9498171F910F91FF90C0
:1030200008951092EE041092ED041092F1041092A3
:103030001E0510921D0514C110921C058091EE040E
:1030400090E02091ED04FC01EE0FFF1FE80FF91F47
:10305000E20FF11DE756FB4F808186FF04C080918F
:10306000F104806803C08091F1048F778093F104AC
:103070000E94C40D8091EE0490E02091ED04FC01CB
:10308000EE0FFF1FE80FF91FE20FF11DE756FB4F90
:10309000808184FF04C08091F104806803C0809126
:1030A000F1048F778093F1040E94C40D8091EE04A7
:1030B00090E02091ED04FC01EE0FFF1FE80FF91FD7
:1030C000E20FF11DE756FB4F808182FF04C0809123
:1030D000F104806803C08091F1048F778093F1043C
:1030E0000E94C40D8091EE0490E02091ED04FC015B
:1030F000EE0FFF1FE80FF91FE20FF11DE756FB4F20
:10310000808180FF04C08091F104806803C08091B9
:10311000F1048F778093F1040E94C40D8091ED0437
:103120008F5F8093ED048091ED04833038F010922E
:10313000ED048091EE048F5F8093EE048091EE04A5
:1031400090E02091ED04FC01EE0FFF1FE80FF91F46
:10315000E20FF11DE756FB4F808186FF04C080918E
:10316000F104806803C08091F1048F778093F104AB
:103170000E94C40D8091EE0490E02091ED04FC01CA
:10318000EE0FFF1FE80FF91FE20FF11DE756FB4F8F
:10319000808184FF04C08091F104806803C0809125
:1031A000F1048F778093F1040E94C40D8091EE04A6
:1031B00090E02091ED04FC01EE0FFF1FE80FF91FD6
:1031C000E20FF11DE756FB4F808182FF04C0809122
:1031D000F104806803C08091F1048F778093F1043B
:1031E0000E94C40D8091EE0490E02091ED04FC015A
:1031F000EE0FFF1FE80FF91FE20FF11DE756FB4F1F
:10320000808180FF04C08091F104806803C08091B8
:10321000F1048F778093F1040E94C40D8091ED0436
:103220008F5F8093ED048091ED04833038F010922D
:10323000ED048091EE048F5F8093EE04E0911D0514
:10324000F0911E0580911C05EE50FB4F808380910C
:103250001D0590911E05019690931E0580931D05F6
:1032600080911D0590911E0589970CF4E5CE84E0B0
:10327000809396058FE280935B0510925C0587E151
:1032800080935D058091090180935E05809195058D
:1032900080935F05109260051092610510921E05E3
:1032A00010921D0517C0A0911D05B0911E05E0915B
:1032B0001D05F0911E05EE50FB4F8081AE59BA4FAF
:1032C0008C9380911D0590911E05019690931E058B
:1032D00080931D0580911D0590911E0589971CF313
:1032E0000E94600F82E390E0909392058093910595
:1032F0000E949817089580912205813109F040C0FD
:1033000080935B0510925C0581E980935D051092C6
:103310005E0594E590935F0583E58093600580E505
:103320008093610588E3809362058EE48093630552
:103330009093640588E48093650580E28093660538
:103340008093670584E48093680586E5809369052A
:103350008DE280936A0590936B0582E580936C05FE
:1033600088E580936D0584E190E0909392058093C9
:1033700091050E94981781E08093990580939705A5
:10338000809122058231E1F485E080935B05109203
:103390005C0582E980935D0583E180935E0589E0A9
:1033A00080935F0580E18093600581E080936105F3
:1033B00088E090E090939205809391050E94981781
:1033C000809122058431D9F580912305803C91F4C8
:1033D0008091250580939C058091260580939D050D
:1033E0008091270580939E058091280580939F05F5
:1033F0000E943B1780912305813C71F480E00E947C
:1034000079250E94BF1280E06EE970E143E050E050
:103410000E9456250E94801682E080935B051092E0
:103420005C0584E980935D0586E080935E0585E018
:1034300090E090939205809391050E949817809157
:1034400022058031D1F4909120059230B1F4809121
:1034500023058093A20590935B0510925C0580E99B
:1034600080935D0586E080935E0585E090E0909313
:103470009205809391050E949817809122058031D2
:1034800069F580912005813049F588E080935B05DE
:1034900010925C0580E980935D0587E480935E056A
:1034A0008091A30580935F058091970580936005C7
:1034B00085E1809361058CEF809362058091A4057E
:1034C000809363058091A505809364058BE090E06F
:1034D00090939205809391050E9498178091220500
:1034E000863139F486E060E00E94012781E0809314
:1034F0009A0580912205873161F58091230580939B
:103500000901809124058093950521E030E0F901BF
:10351000EA5DFA4F8081F901EE50FB4F80832F5F07
:103520003F4F2A32310599F70E945D0E86E590E003
:1035300090937A048093790481E090E090937C04E6
:1035400080937B040E944D0C0E948E0882E0809341
:103550009A0580912205893109F03EC01092AC0590
:103560001092AB05809194058F5F809394058091B4
:103570009405853110F01092940528E030E041E088
:1035800050E0E0917904F0917A04D901A15EBA4F3C
:103590008C91EA5DFE4F80838091790490917A044A
:1035A000019690937A0480937904809179049091A4
:1035B0007A048355934024F050937A04409379041D
:1035C0002F5F3F4F24313105E1F680919A0582301B
:1035D00019F483E080939A05809122058A3109F0DD
:1035E0004DC18091790490917A04019790937A0467
:1035F000809379048091790490917A04892B31F435
:1036000082E593E090937A04809379048091790421
:1036100090917A04019790937A0480937904809131
:10362000790490917A04892B31F482E593E09093A8
:103630007A04809379048091790490917A040197B7
:1036400090937A04809379048091790490917A041C
:10365000892B31F482E593E090937A048093790486
:10366000E0917904F0917A04EA5DFE4F85E580836C
:103670008091790490917A04019690937A048093D2
:1036800079048091790490917A048355934034F0C1
:1036900081E090E090937A0480937904E09179043A
:1036A000F0917A04EA5DFE4F85E58083809179048C
:1036B00090917A04019690937A0480937904809192
:1036C000790490917A048355934034F081E090E03E
:1036D00090937A0480937904E0917904F0917A04CC
:1036E000EA5DFE4F85E580838091790490917A04AC
:1036F000019690937A048093790480917904909153
:103700007A048355934034F081E090E090937A04FA
:1037100080937904E0917904F0917A04EA5DFE4F98
:1037200085E580838091790490917A040196909345
:103730007A04809379048091790490917A04835576
:10374000934034F081E090E090937A048093790480
:10375000E0917904F0917A04EA5DFE4F88EC808371
:103760008091790490917A04019690937A048093E1
:1037700079048091790490917A048355934034F0D0
:1037800081E090E090937A0480937904E091790449
:10379000F0917A04EA5DFE4F8AE780838091790494
:1037A00090917A04019690937A04809379048091A1
:1037B000790490917A048355934034F081E090E04D
:1037C00090937A0480937904E0917904F0917A04DB
:1037D000EA5DFE4F10828091790490917A040196FF
:1037E00090937A04809379048091790490917A047B
:1037F0008355934034F081E090E090937A04809375
:103800007904E0917904F0917A04EA5DFE4F108228
:103810008091790490917A04019690937A04809330
:1038200079048091790490917A048355934034F01F
:1038300081E090E090937A0480937904E091790498
:10384000F0917A04EA5DFE4F1082809179049091A4
:103850007A04019690937A04809379048091790494
:1038600090917A048355934034F081E090E09093F6
:103870007A048093790484E080939A0580912205EC
:103880008F31E1F590912305903CD1F486E080934F
:103890005B0510925C058FE980935D0590935E0552
:1038A00010925F05109260051092610510926205FA
:1038B00089E090E090939205809391050E9498177B
:1038C00090912305913CD1F486E080935B051092A2
:1038D0005C058FE980935D0590935E0510925F050E
:1038E00010926005109261051092620589E090E0E7
:1038F00090939205809391050E94981710921F054E
:10390000109220051092580510925705089583E1F2
:1039100080935B0510925C0589E180935D05809141
:10392000090180935E058091950580935F0588EE7F
:103930008093600583E08093610525E130E04EE1EE
:1039400050E0FA01E21BF30BD901AF57BB4F8C914A
:10395000E75AFA4F8083215030402930310589F7EA
:1039600010926E0510926F0586E190E0909392059B
:10397000809391050E949817089583E080935B05DA
:1039800010925C058AE180935D0580910901809326
:103990005E058091950580935F0586E090E09093A9
:1039A0009205809391050E94981708958F92AF9287
:1039B000BF92CF92EF92FF920F931F932091C80571
:1039C0003091C9054091CA055091CB058091B3054E
:1039D0009091B405A091B505B091B60528173907A7
:1039E0004A075B0709F44FC080E00E9479250E94D6
:1039F000EA100E94801680E06EE970E143E050E03A
:103A00000E9456258091B3059091B405A091B5050B
:103A1000B091B6058093C8059093C905A093CA05D7
:103A2000B093CB058CEC95E00E947F218CEC95E067
:103A30006EE976E00E9443226091C8057091C90545
:103A40008091CA059091CB050E94B62E20E034E209
:103A500044E759E40E94202EAB01BC018CEC95E0B8
:103A600024E00FE017E2EE24FF243EE2C32EAA2456
:103A7000BB24B0E28B2E0E94C7248CEC95E060E65C
:103A800074E00E9443228CEF96E00E94BD28181635
:103A900019060CF500915705109158058CEF96E02A
:103AA0000E94F128015E1A4FF8018083809157052A
:103AB00090915805019690935805809357058091F1
:103AC000570590915805C89734F087E390E090939C
:103AD00058058093570580911F05803D21F0109275
:103AE00058051092570580911F05803D99F48091EB
:103AF00057059091580505976CF020915705309126
:103B000058058091200590E004968217930714F4DD
:103B10000E947B1980919B05813009F045C020915E
:103B2000790430917A0480917B0490917C0482170F
:103B3000930784F48091790490917A0420917B0416
:103B400030917C04821B930B6CE070E00E941E306D
:103B50006093A4052091790430917A0480917B04CC
:103B600090917C042817390794F4809179049091FE
:103B70007A0420917B0430917C048E5A9C4F821BE6
:103B8000930B6CE070E00E941E306093A4052091BE
:103B9000790430917A0480917B0490917C042817F9
:103BA000390711F41092A40580919905882309F42E
:103BB000ECC080919905813009F058C080919A0538
:103BC000882309F453C08AEF90E090930801809312
:103BD00007018CE291E0909306018093050180E05B
:103BE0000E94792581E00E9479258091A3058E7F2E
:103BF0008093A3058091A30582608093A30588E04C
:103C000061E00E9401278DE061E00E9401270E948F
:103C10005F1680E065E175E142E050E00E945625C4
:103C200080919E0525E0829FC00111249093A105FB
:103C30008093A0054091A0055091A10580919F051A
:103C400090E02BEF34E0BC01629FC001639F900DB8
:103C5000729F900D1124840F951F9093A10580935E
:103C6000A00582E08093990580939705809199053E
:103C7000823049F48091A0059091A105059718F430
:103C800083E08093990590919905933061F4809138
:103C90009A05823040F080E48093A80584E0809308
:103CA00099059093970580919905843039F4809116
:103CB000A805823018F485E08093990580919905D4
:103CC000863031F487E08093990585E080939705ED
:103CD00080919905873009F045C08091AB0590919E
:103CE000AC05815C924110F00E9456178091A405AA
:103CF0008530D0F480917B0490917C04CC97909394
:103D00007C0480937B0480917B0490917C04181642
:103D1000190654F080917B0490917C048E5A9C4F3C
:103D200090937C0480937B048091A4058334D0F02D
:103D30008091790490917A04CC9790937A0480933F
:103D400079048091790490917A041816190654F038
:103D50008091790490917A048E5A9C4F90937A04C2
:103D60008093790490919905973049F480919A0550
:103D7000843029F488E08093990590939705809189
:103D80009905893011F40E94561780919605863066
:103D9000C0F52091050130910601809107019091B5
:103DA00008018217930794F480910701909108010C
:103DB0002091050130910601845D9E4F821B930B7B
:103DC0008B3F91051CF081E08093980520910701BD
:103DD00030910801809105019091060182179307A7
:103DE00084F48091070190910801209105013091A0
:103DF0000601821B930B8B3F91051CF081E08093A1
:103E0000980580919805813009F04DC10E94FC0D04
:103E1000809196058823D9F4909198059130B9F452
:103E200080918F048A3A99F480918E048A3A79F4C9
:103E300080918D048A3A59F480918C048A3A39F43D
:103E4000909396058091A30581608093A30580914E
:103E50009605813031F480919805813011F40E94EB
:103E6000B51780919605823061F480919805813074
:103E700041F40E94C70C1092990583E161E00E9411
:103E8000012780919605833031F480919805813027
:103E900011F40E94111880919605843039F48091B4
:103EA0009805813019F485E08093960580919605F8
:103EB0008530D1F4809198058130B1F405C00E941D
:103EC000FC0D809193058F5F8093930580919305FE
:103ED0008131A8F386E0809396051092930584E1E2
:103EE000809394051092980580919605863009F08C
:103EF000DAC080919805813009F0D5C08091930592
:103F00008F5F8093930580919305823008F451C0B0
:103F100080919305893108F04CC0209107013091C0
:103F20000801809105019091060182179307D4F44E
:103F300080910701909108012091050130910601BF
:103F4000821B930B459774F001E010E00E94FC0D7A
:103F5000809193058F5F809393050F5F1F4F013210
:103F60001105A1F720910701309108018091050109
:103F70009091060128173907E4F480910701909188
:103F800008012091050130910601845D9E4F821B3E
:103F9000930B459774F001E010E00E94FC0D8091B6
:103FA00093058F5F809393050F5F1F4F01321105BB
:103FB000A1F7809193058934E1F480918D048535D2
:103FC000C1F480918C048535A1F480918B048535F2
:103FD00081F480918A04853561F480918904883C5C
:103FE00041F4809188048A3721F40E9456170E9478
:103FF000BD1C809194058431A1F480919305823495
:1040000080F080918C04853561F480918B048D3231
:1040100041F480918A04863121F4109298050E941F
:10402000FC0D80919405843119F5809193058934B4
:10403000F9F480918D04853509F042C080918C049B
:104040008D32F1F580918B048631D1F511C08091CC
:104050008C048D3221F080918B048631B1F585E599
:1040600080938D048DE280938C0486E180938B0491
:1040700080919305893431F480919405809395055E
:104080000E94871C80919305803668F010929305FA
:10409000809194058F5F809394058091940585317C
:1040A00010F0109294051092980510929B051F91A4
:1040B0000F91FF90EF90CF90BF90AF908F900895A9
:1040C00080918D04853519F6CACF0E9456170E943B
:1040D000BD1CCECFEF92FF920F931F9382E060E062
:1040E0000E94C22687E061E00E94C22685E060E06F
:1040F0000E94C22686E061E00E94C2268AE061E05A
:104100000E94C2268CE061E00E94C22688E061E045
:104110000E94C2268DE061E00E94C22683E161E038
:104120000E94C22687E060E00E9401278CE060E0E8
:104130000E9401278AE060E00E94012788E060E099
:104140000E9401278DE061E00E9401270CEF16E03C
:10415000C80140E052EC61E070E00E943628C801DE
:104160000E941A290E943B170CEC15E0C80166E476
:1041700070E00E949D23C80161E470E00E94562116
:10418000C80160E070E040E050E028E630E004E57F
:1041900010E0E0E3EE2EF12C0E945F2268E873E16C
:1041A00080E090E00E942E268DE061E00E940127D1
:1041B00080910A0190910B0160E00E94C2268091DB
:1041C0000C0190910D0160E00E94C22680910A01CD
:1041D00090910B0161E00E94012780910C01909168
:1041E0000D0161E00E94012781E063E670E143E098
:1041F00050E00E9456251F910F91FF90EF90089577
:10420000DC011896ED91FC91199790811E968C9186
:104210001E978095892380831496ED91FC911597C4
:10422000442339F490811C968C911C9780958923A6
:1042300005C080811C969C911C97892B808320E06F
:104240001296ED91FC91139767FF06C080811B9633
:104250009C911B97892B06C090811B968C911B9774
:10426000809589238083ED91FC91119790811A9616
:104270008C911A978095892380830000ED91FC91A1
:10428000119780811A969C911A97892B80832F5FB2
:10429000283011F0660FD4CF1896ED91FC91199744
:1042A00080811E969C91892B808308950F931F9384
:1042B000CF93DF938C01EB01603871051CF0CFE7E1
:1042C000D0E004C077FF02C0C0E0D0E0C80161E2E6
:1042D00040E00E940021CE018068682FC80140E0C4
:1042E0000E940021C80160E240E00E940021F80124
:1042F000D28FC18FDF91CF911F910F9108950F93AE
:104300001F93CF93DF938C01FC01808D8823B1F440
:10431000C80160E440E00E940021C80160E840E07C
:104320000E940021C0E0D0E0C80160E041E00E94AE
:1043300000212196F1E0C83FDF07B1F7DF91CF916F
:104340001F910F9108957F928F929F92AF92BF928B
:10435000CF92DF92EF92FF920F931F93CF93DF9351
:10436000EC015901888D882309F07FC08B899A015F
:10437000280F311D253531050CF077C08C898695C5
:10438000869586959501280F311D273031050CF053
:104390006CC0CC24DD2480E8782E742A862E9924E3
:1043A00051C06C2D6A0D6064CE0140E00E94002176
:1043B000CE01672D40E00E9400218C89869586956C
:1043C00086952B89829FC00111242D89A401421B4F
:1043D0005109849F7001859FF00C949FF00C11246B
:1043E00084E090E0E80EF91E00E010E022C08F8922
:1043F000C49E9001C59E300DD49E300D1124E989D4
:10440000FA89882341F42E0D3F1D200F311FE20F42
:10441000F31F649108C02E0D3F1D200F311FE20FC6
:10442000F31F64916095CE0141E00E9400210F5F6F
:104430001F4F8B89482F50E004171507C4F20894CA
:10444000C11CD11C8C8986958695869590E0C816EE
:10445000D9060CF4A6CFCE0160E440E00E94002112
:10446000CE0160E840E00E940021DF91CF911F91D2
:104470000F91FF90EF90DF90CF90BF90AF909F9003
:104480008F907F900895DC01FB0152967C936E9390
:104490005197849153968C93539731968491549667
:1044A0008C9354973196849155968C935597319669
:1044B000E4915696EC93569757961C9208954F9216
:1044C0005F926F927F928F929F92AF92BF92CF92A4
:1044D000DF92EF92FF920F931F93CF93DF934C01E4
:1044E000562EF9013801DC0158968C91882309F089
:1044F0004FC0CA0168E070E00E941E30462EC7011E
:1045000087709070892B39F4C70168E070E00E94D1
:104510001E305B0109C0C70168E070E00E941E30D8
:104520005B010894A11CB11C6F0100E010E0B0E831
:104530005B2A21C0602F640D6064C40140E00E94CA
:104540000021C401652D40E00E9400217601C0E0F9
:10455000D0E00AC0F7016491C40141E00E9400214B
:1045600021960894E11CF11CC615D7059CF30F5F3A
:104570001F4FC60CD71C0A151B05E4F2C40160E4EA
:1045800040E00E940021C40160E840E00E94002158
:10459000DF91CF911F910F91FF90EF90DF90CF901F
:1045A000BF90AF909F908F907F906F905F904F9053
:1045B00008958F929F92AF92BF92CF92DF92EF9227
:1045C000FF920F931F93CF93DF936C015B01E9017F
:1045D000DC0158968C91882309F05AC0DB010D90BC
:1045E0000020E9F78D0101501040061B170BB7E2C0
:1045F0004F305B0779F4F601838990E09C01209F9E
:10460000C001219F900D309F900D112444E550E092
:10461000481B590B37E24E305307A1F4D60153968D
:104620008C9190E0809F9001819F300D909F300D84
:10463000112484E590E0821B930B62E070E00E94FD
:104640001E30AB017A0157FF02C0EE24FF24CE01D9
:1046500068E070E00E941E304B01C0E0D0E015C061
:10466000F50161915F01D60153968C9190E0C89F4E
:10467000A001C99F500DD89F500D11244E0D5F1DF4
:10468000C60194010E94A3212196C017D10744F3CB
:10469000DF91CF911F910F91FF90EF90DF90CF901E
:1046A000BF90AF909F908F9008958F929F92AF92FE
:1046B000BF92CF92DF92EF92FF920F931F93DF93FF
:1046C000CF93CDB7DEB77C01FB016A0159018DB6EE
:1046D0009EB6448155814F5F5F4F8DB79EB7841B57
:1046E000950B0FB6F8949EBF0FBE8DBF0DB71EB7CA
:1046F0000F5F1F4FD70158968C91882361F4CB012F
:10470000B80120E030E00E94FC29C701B801A601F1
:1047100095010E94D9220FB6F8949EBE0FBE8DBEA1
:10472000CF91DF911F910F91FF90EF90DF90CF908D
:10473000BF90AF909F908F900895EF92FF920F934C
:104740001F93CF93DF93EC017B016038710524F058
:104750009FE7E92EF12C04C077FF02C0EE24FF246E
:10476000EC81FD8180819C85892B8083EA81FB819E
:1047700080819B85892B8083E881F98180819A855E
:10478000892B8083E885F98580819E85892B8083AC
:10479000EE81FF8190818D858095892380836AE0F9
:1047A00070E080E090E00E942E26EE81FF81808103
:1047B0009D85892B8083CE0161E240E00E9400212B
:1047C0006E2D6068CE0140E00E940021CE0166E0BF
:1047D00040E00E940021CE0163E140E00E94002100
:1047E000CE0160E240E00E940021CE0160E440E0A2
:1047F0000E940021CE0160E840E00E94002100E01C
:1048000010E0CE0160E041E00E9400210F5F1F4FE9
:1048100081E0083F1807A9F7CE016CE040E00E9454
:1048200000211A8A198A188EFA8EE98EDF91CF91AB
:104830001F910F91FF90EF9008956F927F929F923A
:10484000AF92BF92CF92DF92EF92FF920F931F939E
:10485000CF93DF936C01B62EA42E922EA62FB72FE6
:104860002EE1622E2AE0722EF301EA0FFB1FE49183
:10487000F0E0EE0FFF1F6AE07AE0E60FF71F859188
:104880009491F60191838083C2E3DAE0AC0FBD1FFF
:10489000FD018491F6018287A42FB52FF301EA0F61
:1048A000FB1FE491F0E0EE0FFF1FE60FF71F85916D
:1048B0009491F60193838283AC0FBD1FFD01549147
:1048C000F6015387492D532FF301E40FF51FE491AF
:1048D000F0E0EE0FFF1FE60FF71F85919491F601B0
:1048E000958384834C0F5D1FFA013491F601348760
:1048F0009801F301E00FF11FE491F0E0EE0FFF1FCC
:10490000E60FF71F85919491F601978386832C0F0C
:104910003D1FF9011491F60115876E0C7F1CF30100
:104920008491E82FF0E0EE0FFF1FE60FF71F85914F
:104930009491F60191878087CE0DDF1DFE01849151
:10494000F60186878B2D61E00E94C2268A2D61E0E8
:104950000E94C226892D61E00E94C226802F61E05C
:104960000E94C2268E2D61E00E94C226F601B78603
:10497000008BDF91CF911F910F91FF90EF90DF900F
:10498000CF90BF90AF909F907F906F9008952F929F
:104990003F924F925F926F927F928F92AF92CF929F
:1049A000DF92EF92FF920F931F93DF93CF93CDB7D8
:1049B000DEB76F970FB6F894DEBF0FBECDBF1C01F8
:1049C0002A013B011D8F0C8FFF8EEE8EDC2CC82C34
:1049D000FC01808D882309F052C0CB01BA014A2D19
:1049E0007E010894E11CF11C87010E94D605FEE2BD
:1049F000DF1669F0F7019E01245E3F4F05C08081FC
:104A00008E3209F4D0823196E217F307C1F780E2C3
:104A1000C81659F1C301B20120E030E040E050E097
:104A20000E941C2E87FD06C0FE0131969E01245E69
:104A30003F4F18C08DE28983FE0132969E01245EAD
:104A40003F4F07C08081803211F08D3209F4C0825F
:104A50003196E217F307B1F708C08081803209F47C
:104A6000C0823196E217F307C1F7C101BE016F5F43
:104A70007F4F4C8D5D8D2E8D3F8D0E94D9226F967C
:104A80000FB6F894DEBF0FBECDBFCF91DF911F915F
:104A90000F91FF90EF90DF90CF90AF908F907F902D
:104AA0006F905F904F903F902F900895823000F567
:104AB000E82FF0E0EE0FFF1FE951FA4F718360839A
:104AC000882319F08130A1F408C0809169008C7F9F
:104AD000842B80936900E89A089580916900440FBF
:104AE000551F440F551F837F842B80936900E99ADB
:104AF0000895823080F4882319F0813021F402C0B7
:104B0000E89801C0E998E82FF0E0EE0FFF1FE951A7
:104B1000FA4F1182108208951F920F920FB60F92D2
:104B200011242F933F934F935F936F937F938F93B2
:104B30009F93AF93BF93EF93FF938091E70590917D
:104B4000E805892B29F0E091E705F091E805099542
:104B5000FF91EF91BF91AF919F918F917F916F9155
:104B60005F914F913F912F910F900FBE0F901F902B
:104B700018951F920F920FB60F9211242F933F9307
:104B80004F935F936F937F938F939F93AF93BF9355
:104B9000EF93FF938091E9059091EA05892B29F025
:104BA000E091E905F091EA050995FF91EF91BF9138
:104BB000AF919F918F917F916F915F914F913F91B5
:104BC0002F910F900FBE0F901F9018951F920F926C
:104BD0000FB60F9211242F933F938F939F93AF9310
:104BE000BF938091EF059091F005A091F105B091F0
:104BF000F2053091F3050196A11DB11D232F2D5F04
:104C00002D3720F02D570196A11DB11D2093F305DE
:104C10008093EF059093F005A093F105B093F20512
:104C20008091EB059091EC05A091ED05B091EE051A
:104C30000196A11DB11D8093EB059093EC05A09307
:104C4000ED05B093EE05BF91AF919F918F913F918C
:104C50002F910F900FBE0F901F9018959B01AC01E4
:104C60007FB7F8948091EB059091EC05A091ED054C
:104C7000B091EE0566B5A89B05C06F3F19F001968F
:104C8000A11DB11D7FBFBA2FA92F982F8827860F8E
:104C9000911DA11DB11D62E0880F991FAA1FBB1FA6
:104CA0006A95D1F7BC012DC0FFB7F8948091EB0550
:104CB0009091EC05A091ED05B091EE05E6B5A89BAD
:104CC00005C0EF3F19F00196A11DB11DFFBFBA2F1E
:104CD000A92F982F88278E0F911DA11DB11DE2E0ED
:104CE000880F991FAA1FBB1FEA95D1F7861B970B48
:104CF000885E9340C8F22150304040405040685197
:104D00007C4F211531054105510571F608957894C0
:104D100084B5826084BD84B5816084BD85B58260C0
:104D200085BD85B5816085BDEEE6F0E0808181605E
:104D30008083E1E8F0E0108280818260808380815E
:104D400081608083E0E8F0E0808181608083E1EB36
:104D5000F0E0808184608083E0EBF0E0808181601E
:104D60008083EAE7F0E080818460808380818260D4
:104D700080838081816080838081806880831092BD
:104D8000C1000895CF93DF93482F50E0CA018E5C95
:104D9000954FFC013491425E554FFA01849188236E
:104DA00069F190E0880F991FFC01E050F64FA59142
:104DB000B491FC01E65FF54FC591D491662351F49F
:104DC0002FB7F8948C91932F909589238C93888199
:104DD00089230BC0623061F42FB7F8948C91932F24
:104DE000909589238C938881832B88832FBF06C05D
:104DF0009FB7F8948C91832B8C939FBFDF91CF91B9
:104E00000895482F50E0CA018A5B954FFC01249118
:104E1000CA018E5C954FFC019491425E554FFA0198
:104E20003491332309F440C0222351F1233071F02F
:104E3000243028F42130A1F0223011F514C026309E
:104E4000B1F02730C1F02430D9F404C08091800043
:104E50008F7703C0809180008F7D8093800010C089
:104E600084B58F7702C084B58F7D84BD09C08091E1
:104E7000B0008F7703C08091B0008F7D8093B00029
:104E8000E32FF0E0EE0FFF1FE65FF54FA591B49121
:104E90002FB7F894662321F48C919095892302C052
:104EA0008C91892B8C932FBF0895682F70E0CB01D4
:104EB0008A5B954FFC012491CB018E5C954FFC01E0
:104EC0004491625E754FFB019491992319F420E09F
:104ED00030E03CC0222351F1233071F0243028F41B
:104EE0002130A1F0223011F514C02630B1F0273066
:104EF000C1F02430D9F404C0809180008F7703C0C2
:104F0000809180008F7D8093800010C084B58F7762
:104F100002C084B58F7D84BD09C08091B0008F77B9
:104F200003C08091B0008F7D8093B000892F90E006
:104F3000880F991F8C5E954FFC01A591B4918C91BF
:104F400020E030E0842311F021E030E0C901089531
:104F500008951F920F920FB60F9211242F933F9333
:104F60004F938F939F93EF93FF938091C00082FDA7
:104F70001DC04091C60020917406309175062F5FC8
:104F80003F4F2F77307080917606909177062817E3
:104F9000390771F0E0917406F0917506EC50FA4F04
:104FA0004083309375062093740602C08091C6003A
:104FB000FF91EF919F918F914F913F912F910F9082
:104FC0000FBE0F901F901895E0910807F091090708
:104FD000E058FF4F819191912081318180589F4FFE
:104FE000821B930B60E870E00E941E30892B11F049
:104FF0000E94A82708951F920F920FB60F921124B6
:105000002F933F938F939F93EF93FF932091F806F5
:105010003091F9068091FA069091FB06281739071E
:1050200031F48091C1008F7D8093C10014C0E09164
:10503000FA06F091FB06E858F94F20818091FA06B4
:105040009091FB0601968F7790709093FB0680936A
:10505000FA062093C600FF91EF919F918F913F91A7
:105060002F910F900FBE0F901F901895AF92BF9287
:10507000DF92EF92FF920F931F93CF93DF93EC0198
:105080007A018B01DD24403081EE580780E068070B
:1050900080E0780711F0DD24D39491E0A92EB12CA3
:1050A000EC89FD89DD2069F0C50108A002C0880FE8
:1050B000991F0A94E2F7808360E079E08DE390E045
:1050C00005C0108260E874E88EE190E0A8019701C5
:1050D0000E94313021503040404050405695479515
:1050E0003795279580E12030380720F0DD2011F03A
:1050F000DD24D6CFE889F9893083EA89FB892083CA
:1051000019A2EE89FF89408121E030E0C9010C8CB1
:1051100002C0880F991F0A94E2F7482B4083EE895A
:10512000FF894081C9010D8C02C0880F991F0A9424
:10513000E2F7482B4083EE89FF894081C9010E8C3C
:1051400002C0880F991F0A94E2F7482B4083EE892A
:10515000FF8980810F8C02C0220F331F0A94E2F76F
:10516000209528232083DF91CF911F910F91FF90ED
:10517000EF90DF90BF90AF900895DC011C96ED9109
:10518000FC911D97E058FF4F8191919120813181D1
:1051900080589F4F821B930B60E870E00E941E3086
:1051A0000895DC011C96ED91FC911D97E058FF4F8E
:1051B00020813181E058F040DF01AE57BF4F8D9123
:1051C0009C9111972817390719F42FEF3FEF07C06B
:1051D0008D919C91E80FF91F8081282F30E0C90143
:1051E0000895DC011C96ED91FC911D97E058FF4F4E
:1051F00020813181E058F040DF01AE57BF4F8D91E3
:105200009C9111972817390719F42FEF3FEF10C021
:105210008D919C911197E80FF91F20818D919C91A0
:10522000119701968F77907011969C938E9330E032
:10523000C9010895DC0191968C919197882339F0EA
:105240005496ED91FC915597808186FFF9CF919608
:105250001C920895CF93DF93EC01EE85FF85E05813
:10526000FF4F20813181E058F0402F5F3F4F2F7773
:105270003070DF01AE57BF4F8D919C911197281769
:105280003907D1F3E058FF4F80819181E058F04019
:10529000E80FF91F6083EE85FF85E058FF4F3183EB
:1052A0002083EE89FF89208181E090E00F8C02C08D
:1052B000880F991F0A94E2F7282B208381E089A3A5
:1052C000EC89FD8980818064808381E090E0DF91BA
:1052D000CF9108951092FF061092FE0688EE93E09B
:1052E000A0E0B0E08093000790930107A09302072D
:1052F000B093030788E191E09093FD068093FC064C
:1053000084EF95E0909309078093080788E796E07B
:1053100090930B0780930A0785EC90E090930D071C
:1053200080930C0784EC90E090930F0780930E0716
:1053300080EC90E0909311078093100781EC90E04F
:10534000909313078093120782EC90E090931507D7
:105350008093140786EC90E09093170780931607CC
:1053600084E08093180783E08093190787E0809397
:105370001A0785E080931B0781E080931C0708953E
:105380000895CF93DF930E9487260E94C0290E9430
:105390006A20C4EED7E20E94D61C2097E1F30E9457
:1053A000E427F9CFCF92DF92EF92FF920F931F93F2
:1053B000CF93DF937C016B018A01C0E0D0E00FC086
:1053C000D6016D916D01D701ED91FC910190F081B5
:1053D000E02DC7010995C80FD91F015010400115D4
:1053E000110571F7CE01DF91CF911F910F91FF90C1
:1053F000EF90DF90CF9008950F931F93CF93DF939B
:10540000FC018B0141155105F9F061157105E1F0C1
:10541000848195812817390718F0FB01108214C088
:1054200041505040EC01C21BD30B4C175D0708F4F0
:10543000EA0160817181620F731FC801AE010E9491
:105440000706C00FD11F1882DF91CF911F910F91D6
:1054500008950F931F93CF93DF93EC018B016F5F40
:105460007F4F888199810E94D62C009711F480E0AB
:1054700005C0998388831B830A8381E0DF91CF91E4
:105480001F910F910895CF93DF93EC01888199814B
:10549000892B29F08A819B818617970760F4CE01BA
:1054A0000E94292A882341F08C819D81892B19F43F
:1054B000E881F981108281E0DF91CF910895EF9228
:1054C000FF920F931F93CF93DF93EC017B016C81CD
:1054D0007D81E114F104C1F04115510599F08A0173
:1054E000060F171FB8010E94432A882369F088819C
:1054F00099812C813D81820F931FB7010E94000684
:105500001D830C8381E001C080E0DF91CF911F916A
:105510000F91FF90EF900895CF93DF93EC01888176
:105520009981009711F00E943E2C198218821D82E9
:105530001C821B821A82DF91CF9108950F931F93D3
:10554000182F092F6115710561F0DB010D90002006
:10555000E9F71197A61BB70BAD010E945F2A8823BC
:1055600021F4812F902F0E948C2A812F902F1F9140
:105570000F9108950F931F93182F092FFB0160813E
:105580007181448155810E945F2A882321F4812FF3
:10559000902F0E948C2A812F902F1F910F91089598
:1055A000EF92FF920F931F93CF93DF93EC017B0158
:1055B0008A01BA010E94432A882321F4CE010E9465
:1055C0008C2A07C01D830C8388819981B7010E94B2
:1055D0000006CE01DF91CF911F910F91FF90EF90C8
:1055E0000895CF93DF93EC01198218821B821A82EF
:1055F0001D821C826115710551F0DB010D900020A8
:10560000E9F71197A61BB70BAD010E94D02ADF91D5
:10561000CF9108950F931F93182F092F61157105CE
:1056200059F0DB010D900020E9F71197A61BB70B8D
:10563000AD010E94D02A02C00E948C2A812F902F97
:105640001F910F910895BF92CF92DF92EF92FF9238
:105650000F931F93CF93DF93082FB92E6B017A011D
:10566000E9012417350710F4EA017901802F9B2DF9
:1056700064E071E00E94F12AD60114968D919C910C
:1056800015978E159F05D0F08C179D0708F4EC0137
:10569000D601ED91FC911197EC0FFD1F1081108246
:1056A0006D917C916E0D7F1D802F9B2D0E940A2B8A
:1056B000D601ED91FC91EC0FFD1F1083802F9B2DE7
:1056C000DF91CF911F910F91FF90EF90DF90CF90DE
:1056D000BF900895CF93DF93EC01FB0186179707E6
:1056E00061F0608171816115710529F044815581F6
:1056F0000E94D02A02C00E948C2ACE01DF91CF9155
:105700000895FC0111821082138212821582148284
:105710000E946A2B0895FC0111821082138212826A
:10572000158214820E946A2B0895FC018081918168
:105730000E943E2C0895FC01808191810E943E2CA4
:1057400008950F931F93CF93DF93BC01823091058F
:1057500010F462E070E0E0912007F091210740E052
:1057600050E0A0E0B0E024C08081918186179707C7
:10577000D0F08617970771F482819381109729F0F2
:1057800013969C938E9312972CC09093210780932D
:10579000200727C04115510519F08417950718F403
:1057A0008D01AC01EF01DF01828193819C01F90140
:1057B0003097D1F641155105F9F0CA01861B970BB8
:1057C0008430910580F48A819B810115110521F0B7
:1057D000F8019383828304C090932107809320076C
:1057E000FE01329645C0FE01E80FF91F61937193E7
:1057F0000297998388833CC080911E0790911F0770
:10580000892B41F4809110019091110190931F0711
:1058100080931E07409112015091130141155105CB
:1058200041F44DB75EB780910E0190910F01481B76
:10583000590B20911E0730911F0724173507B0F42C
:10584000CA01821B930B8617970780F0AB014E5F4E
:105850005F4F8417950750F0420F531F50931F0757
:1058600040931E07F9016193719302C0E0E0F0E0FC
:10587000CF01DF91CF911F910F910895CF93DF93C7
:105880009C01009709F48FC0EC0122971B821A82B9
:1058900060912007709121076115710581F488815D
:1058A0009981820F931F20911E0730911F0728179F
:1058B000390739F5D0931F07C0931E0774C0DB0169
:1058C00040E050E0AC17BD0708F1BB83AA83FE019E
:1058D00021913191E20FF31FAE17BF0779F48D913B
:1058E0009C911197280F391F2E5F3F4F39832883D2
:1058F00012968D919C9113979B838A834115510534
:1059000071F4D0932107C09320074DC012968D915A
:105910009C911397AD01009711F0DC01D3CFDA0110
:105920001396DC93CE931297FA0121913191E20FF5
:10593000F31FCE17DF0769F488819981280F391F7B
:105940002E5F3F4FFA01318320838A819B819383AD
:105950008283E0E0F0E0DB0112968D919C91139739
:10596000009719F0BC01FD01F6CFAB014E5F5F4F10
:10597000DB018D919C91840F951F20911E07309122
:105980001F072817390779F4309729F41092210757
:105990001092200702C0138212824250504050934E
:1059A0001F0740931E07DF91CF9108956F927F925A
:1059B0008F929F92AF92BF92CF92DF92EF92FF921F
:1059C0000F931F93CF93DF938C01009729F4CB01A2
:1059D0000E94A12B8C01BBC08EEFE82E8FEFF82E1A
:1059E000E00EF11E4801860E971E8E149F0408F4E7
:1059F000ACC0D7014D915C91119746175707B8F08D
:105A00004530510508F4A3C0CA01049786179707CB
:105A100008F49DC042505040461B570BF40141937F
:105A200051936D937C93CF010E943E2C90C05B01FB
:105A3000A41AB50A3801640E751EA0912007B09112
:105A40002107E0E0F0E0CC24DD2447C0A615B7052F
:105A5000A9F5CD91DC911197CE0102968A159B058F
:105A600068F1CE018A199B09029612962C91129721
:105A700013963C91059758F0F40122833383CA1999
:105A8000DB09D183C083D7016D937C9309C04E5F3E
:105A90005F4F4C0F5D1FF70151834083C901FC012B
:105AA000C114D10431F0D6011396FC93EE931297F2
:105AB0004EC0F0932107E093200749C08D919C913F
:105AC0001197E817F90708F4FC016D0112968C9103
:105AD000129713969C919C01D901109709F0B6CFAB
:105AE00080911E0790911F0786159705E9F4E61728
:105AF000F707D0F4209112013091130121153105DF
:105B000041F42DB73EB780910E0190910F01281BF3
:105B1000390B82169306C8F490921F0780921E07D5
:105B2000F7017183608313C0CB010E94A12BEC01AC
:105B3000009759F0D7014D915C91B8010E94F7058B
:105B4000C8010E943E2C8E0102C000E010E0C80196
:105B5000DF91CF911F910F91FF90EF90DF90CF9049
:105B6000BF90AF909F908F907F906F900895505806
:105B7000BB27AA270ED0AEC19FD130F0A4D120F010
:105B800031F49F3F11F41EF494C10EF4E095E7FB4D
:105B90005FC1E92FB0D180F3BA176207730784079A
:105BA000950718F071F49EF5DFC10EF4E0950B2E09
:105BB000BA2FA02D0B01B90190010C01CA01A0015F
:105BC0001124FF27591B99F0593F50F4503E68F1BA
:105BD0001A16F040A22F232F342F4427585FF3CFFB
:105BE000469537952795A795F0405395C9F77EF4CC
:105BF0001F16BA0B620B730B840BBAF09150A1F015
:105C0000FF0FBB1F661F771F881FC2F70EC0BA0F9A
:105C1000621F731F841F48F4879577956795B79522
:105C2000F7959E3F08F0B3CF9395880F08F099271A
:105C3000EE0F979587950895E7D008F481E00895D1
:105C40000CD048C140D140F037D130F021F45F3F53
:105C500019F0FEC0511189C12CC14DD198F399237F
:105C6000C9F35523B1F3951B550BBB27AA27621720
:105C70007307840738F09F5F5F4F220F331F441F65
:105C8000AA1FA9F333D00E2E3AF0E0E830D091509D
:105C90005040E695001CCAF729D0FE2F27D0660F8A
:105CA000771F881FBB1F261737074807AB07B0E8C9
:105CB00009F0BB0B802DBF01FF2793585F4F2AF0DF
:105CC0009E3F510568F0C4C050C15F3FECF3983E61
:105CD000DCF3869577956795B795F7959F5FC9F73C
:105CE000880F911D9695879597F90895E1E0660FC5
:105CF000771F881FBB1F621773078407BA0720F03E
:105D0000621B730B840BBA0BEE1F88F7E0950895A6
:105D1000FAD088F09F5790F0B92F9927B751A0F08B
:105D2000D1F0660F771F881F991F1AF0BA95C9F72F
:105D300012C0B13081F018D1B1E0089515C1672FBC
:105D4000782F8827B85F39F0B93FCCF386957795DF
:105D50006795B395D9F73EF49095809570956195C8
:105D60007F4F8F4F9F4F0895E89409C097FB3EF4F3
:105D700090958095709561957F4F8F4F9F4F992398
:105D8000A9F0F92F96E9BB279395F6958795779516
:105D90006795B795F111F8CFFAF4BB0F11F460FFD6
:105DA0001BC06F5F7F4F8F4F9F4F16C0882311F02E
:105DB00096E911C0772321F09EE8872F762F05C042
:105DC000662371F096E8862F70E060E02AF09A95DD
:105DD000660F771F881FDAF7880F9695879597F9D2
:105DE0000895ABD080F09F3740F491110EF0BDC004
:105DF00060E070E080E89FEB089526F41B16611DBB
:105E0000711D811D2BC045C0990F0008550FAA0BAD
:105E1000E0E8FEEF16161706E807F907C0F01216BD
:105E20001306E407F50798F0621B730B840B950BC0
:105E300039F40A2661F0232B242B252B21F4089515
:105E40000A2609F4A140A6958FEF811D811D0895B2
:105E500097F99F6780E870E060E00895882371F407
:105E6000772321F09850872B762F07C0662311F4F3
:105E700099270DC09051862B70E060E02AF09A952A
:105E8000660F771F881FDAF7880F9695879597F921
:105E900008959F3F49F0915028F48695779567952E
:105EA000B7959F5F80389F4F880F9695879597F994
:105EB00008959FEF80EC089500240A9416161706A3
:105EC00018060906089500240A94121613061406EB
:105ED00005060895092E0394000C11F4882352F04E
:105EE000BB0F40F4BF2B11F460FF04C06F5F7F4F06
:105EF0008F4F9F4F089557FD9058440F551F59F0ED
:105F00005F3F71F04795880F97FB991F61F09F3FA6
:105F100079F087950895121613061406551FF2CFCF
:105F20004695F1DF08C0161617061806991FF1CF1F
:105F300086957105610508940895E5DFA0F0BEE738
:105F4000B91788F4BB279F3860F41616B11D672F68
:105F5000782F8827985FF7CF869577956795B11D3D
:105F600093959639C8F30895E894BB276627772759
:105F7000CB0197F908950BD0ADCF9EDF28F0A3DFBA
:105F800018F0952309F064CF94CF1124EECFB3DF3E
:105F9000A0F3959FD1F3950F50E0551F629FF0013C
:105FA000729FBB27F00DB11D639FAA27F00DB11D95
:105FB000AA1F649F6627B00DA11D661F829F22271E
:105FC000B00DA11D621F739FB00DA11D621F839FA5
:105FD000A00D611D221F749F3327A00D611D231F7B
:105FE000849F600D211D822F762F6A2F11249F57C9
:105FF00050408AF0E1F088234AF0EE0FFF1FBB1FEC
:10600000661F771F881F91505040A9F79E3F51058A
:1060100070F01ECFAACF5F3FECF3983EDCF386957D
:1060200077956795B795F795E7959F5FC1F7FE2B35
:10603000880F911D9695879597F9089597FB092EDE
:1060400007260AD077FD04D02ED006D000201AF4FF
:10605000709561957F4F0895F6F7909581959F4FC4
:106060000895A1E21A2EAA1BBB1BFD010DC0AA1F99
:10607000BB1FEE1FFF1FA217B307E407F50720F0B1
:10608000A21BB30BE40BF50B661F771F881F991F2C
:106090001A9469F760957095809590959B01AC0175
:1060A000BD01CF010895AA1BBB1B51E107C0AA1F68
:1060B000BB1FA617B70710F0A61BB70B881F991FA9
:1060C0005A95A9F780959095BC01CD010895EE0FE2
:1060D000FF1F0590F491E02D09942F923F924F926B
:1060E0005F926F927F928F929F92AF92BF92CF9268
:1060F000DF92EF92FF920F931F93CF93DF93CDB771
:10610000DEB7CA1BDB0B0FB6F894DEBF0FBECDBFE8
:1061100009942A88398848885F846E847D848C84B9
:106120009B84AA84B984C884DF80EE80FD800C81C2
:106130001B81AA81B981CE0FD11D0FB6F894DEBFA5
:0C6140000FBECDBFED010895F894FFCF15
:10614C00203E2000002C01FA000103001500800005
:10615C0022070000000000002A29D229BD28F128BE
:04616C00D1281A29F3
:00000001FF
